:100000000C9456050C9473050C9473050C947305AD
:100010000C9473050C9473050C9473050C94730580
:100020000C9473050C9473050C9484250C94582639
:100030000C94BC1F0C9473050C9473050C947305FD
:100040000C9473050C9473050C9473050C94730550
:100050000C9473050C9443200C9473050C94730555
:100060000C9473050C9473050C9473050C94730530
:100070000C9473050C9473050C9473050C94730520
:100080000C9473050C9473050C9473050C94730510
:100090000C9473050C9473050C9473050C94730500
:1000A0000C9473050C9473050C947305165C1E0078
:1000B0001F0020002100220023002400250026002C
:1000C00027002D002E002A0035002B0014001A00F6
:1000D0000800150017001C0018000C001200130087
:1000E0002F00300031004C003900040016000700DA
:1000F00009000A000B000D000E000F003300340051
:10010000000028004B00E10000001D001B0006005D
:100110001900050011001000360037003800E50016
:1001200052004E00E0000151E2000000000000001B
:100130002C000000000004000500060050005100E3
:100140004F0001003A003B003C003D003E003F00F4
:100150004000410042004300440045004C000000C4
:100160000100010052000100010001000100010036
:10017000010001000100010001000100490001002F
:10018000500051004F00010001000100010001007A
:10019000010001000100000001004A000100000010
:1001A00001000100BE5CC05CBF5C0100AA00A900A8
:1001B000A8000100F100ED004D0001000100010068
:1001C000000000000000010000000000010001002C
:1001D0000100EF00EE00F00044454255473A20642C
:1001E000697361626C65642E0A0044454255473A62
:1001F00020656E61626C65642E0A000A002530324B
:1002000058006C65645F7461736B3A20004F6E65D3
:1002100073686F743A206163746976653A20256467
:100220000A000A002530313662003A2000253032BB
:1002300058000A722F632030313233343536373864
:10024000394142434445460A00290A002575002FDA
:10025000002575005D28002564002000256400202D
:100260000025640020002564007C00253032580001
:100270006D6F7573656B6579205B62746E7C782039
:1002800079207620685D287265702F61636C293A49
:10029000205B00313A0964656C6179282A31306D40
:1002A00073293A2025750A323A09696E74657276A7
:1002B000616C286D73293A2025750A333A096D61FE
:1002C000785F73706565643A2025750A343A09745D
:1002D000696D655F746F5F6D61783A2025750A35C9
:1002E0003A09776865656C5F6D61785F7370656505
:1002F000643A2025750A363A09776865656C5F743B
:10030000696D655F746F5F6D61783A2025750A00CD
:10031000703A097072696E742076616C7565730A43
:10032000643A097365742064656661756C74730A58
:1003300075703A092B310A646E3A092D310A6C74D2
:100340003A092B31300A72743A092D31300A45537B
:10035000432F713A09717569740A0A73706565648F
:10036000203D2064656C7461202A206D61785F7384
:1003700070656564202A2028726570656174202F7D
:100380002074696D655F746F5F6D6178290A7768A5
:100390006572652064656C74613A20637572736F71
:1003A000723D25642C20776865656C3D25640A5391
:1003B000656520687474703A2F2F656E2E77696BAF
:1003C0006970656469612E6F72672F77696B692F39
:1003D0004D6F7573655F6B6579730A004D3E200044
:1003E0004D25753A25733E20003F0A003D202575B6
:1003F0000A003F0A0064656661756C74730A002523
:10040000750A003F0A000A092D2056616C75657354
:10041000202D0A00710A000A092D204D6F757365A1
:100420006B6579202D0A003F00433E20004C256477
:100430000A000A092D20537461747573202D0A680F
:100440006F73745F6B6579626F6172645F6C656412
:100450007328293A20253032580A6B6579626F611A
:1004600072645F70726F746F636F6C3A2025303204
:10047000580A6B6579626F6172645F69646C653A92
:1004800020253032580A74696D65725F7265616447
:10049000333228293A202530386C580A000A092DB1
:1004A0002056657273696F6E202D0A5649443A20B2
:1004B00030783545363828756D62796E6F7329202E
:1004C0005049443A20307835463030287369636BA0
:1004D000363829205645523A203078303030310AAB
:1004E0004255494C443A2020284A756E2020372036
:1004F00032303232290A4F5054494F4E533A204C31
:10050000554641204D4F5553454B4559204558546C
:1005100052414B455920434F4E534F4C4520434F7A
:100520004D4D414E4420343039360A4743433A203A
:10053000382E332E30204156522D4C4942433A201A
:10054000322E302E30204156525F415243483A20DD
:10055000617672350A000A092D20436F6E736F6C45
:1005600065202D0A4553432F713A09717569740A44
:100570006D3A096D6F7573656B65790A000A092D0F
:10058000204D61676963202D0A443A09446562750C
:1005900067204D65737361676520546F67676C658D
:1005A0000A583A094D61747269782044656275672A
:1005B000204D6F646520546F67676C65202D205354
:1005C000686F77206B6579707265737365732069E6
:1005D0006E206D617472697820677269640A4B3AA3
:1005E000094B6579626F61726420446562756720AA
:1005F000546F67676C65202D2053686F77206B659B
:10060000797072657373207265706F72740A4D3AF7
:10061000094465627567204D6F75736520546F6777
:10062000676C650A563A0956657273696F6E0A53AC
:100630003A095374617475730A433A0941637469E2
:100640007661746520436F6E736F6C65204D6F64C7
:10065000650A46312D4631303A095377697463682B
:1006600020746F204C6179657220302D3920284626
:100670003130203D204C30290A302D393A0953774A
:100680006974636820746F204C6179657220302D25
:10069000390A47524156453A0953776974636820CD
:1006A000746F204C6179657220302028616C74650C
:1006B000726E617465290A423A094A756D70207438
:1006C0006F20426F6F746C6F616465720A455343AB
:1006D0003A094A756D7020746F20426F6F746C6FA9
:1006E000616465722028616C7465726E617465293D
:1006F0000A453A095072696E7420454550524F4D73
:100700002053657474696E67730A425350414345C0
:100710003A09436C65617220454550524F4D0A00BD
:100720006B65796D61705F636F6E6669672E72616C
:10073000773A20253032580A2E737761705F636FE5
:100740006E74726F6C5F636170736C6F636B3A2071
:1007500025750A2E636170736C6F636B5F746F5FD6
:10076000636F6E74726F6C3A2025750A2E73776111
:10077000705F6C63746C5F6C6775693A2025750AED
:100780002E737761705F7263746C5F726775693A1C
:100790002025750A2E737761705F6C616C745F6CD5
:1007A0006775693A2025750A2E737761705F7261EB
:1007B0006C745F726775693A2025750A2E6E6F5FDB
:1007C0006775693A2025750A2E737761705F6772C5
:1007D0006176655F6573633A2025750A2E737761CC
:1007E000705F6261636B736C6173685F6261636B9E
:1007F00073706163653A2025750A2E6E6B726F3ACD
:100800002025750A0064656275675F636F6E6669AF
:10081000672E7261773A20253032580A2E656E6154
:10082000626C653A2025750A2E6D61747269783A9A
:100830002025750A2E6B6579626F6172643A2025F6
:10084000750A2E6D6F7573653A2025750A0065650A
:10085000636F6E6669673A0A64656661756C745F9A
:100860006C617965723A2025750A003F000A6D6F48
:100870007573653A206F66660A000A6D6F75736559
:100880003A206F6E0A000A6B6579626F6172643A92
:10089000206F66660A000A6B6579626F6172643A5E
:1008A000206F6E0A000A6D61747269783A206F6673
:1008B000660A000A6D61747269783A206F6E0A00E8
:1008C0000A64656275673A206F66660A000A6465A5
:1008D0006275673A206F6E0A000A0A4A756D706980
:1008E0006E6720746F20626F6F746C6F61646572E5
:1008F0002E2E2E2000433E2000436C656172696EEF
:100900006720454550524F4D0A000A0025303258A5
:1009100020006B6579626F6172645F7265706F72DF
:10092000743A20005B735D005B575D005B535D00B4
:100930005B525D005B445D005B435D000E03730032
:10094000690063006B00360038000000100375007A
:100950006D00620079006E006F00730000000403F8
:10096000090409025B00030100A0FA090400000168
:100970000301010009211101000122400007058146
:10098000030800010904010001030000000921110E
:10099000010001227B0007058203200001090402F7
:1009A00000020300000009211101000122220007BA
:1009B0000583032000010705030320000112010045
:1009C0000200000008685E005F01000102000106ED
:1009D00031FF0974A1010975150026FF00952075E6
:1009E0000881020976150026FF00952075089102FE
:1009F000C005010902A10185020901A1000509192B
:100A000001290815002501950875018102050109D4
:100A10003009311581257F95027508810609381541
:100A200081257F950175088106050C0A380215811C
:100A3000257F950175088106C0C005010980A101C7
:100A4000850319012AB700150126B7009501751015
:100A50008100C0050C0901A101850419012AA00229
:100A6000150126A002950175108100C00501090637
:100A7000A101050719E029E7150025019508750171
:100A800081029501750881010507190029FF1500EC
:100A900026FF0095067508810005081901290595AE
:100AA0000575019102950175039101C011241FBEC6
:100AB000CFEFDAE0DEBFCDBF11E0A0E0B1E0ECEABD
:100AC000F1E502C005900D92AA3FB107D9F722E0E7
:100AD000AAEFB1E001C01D92A03FB207E1F70E946A
:100AE0005B160C94BE280C940000FF93EF93E091EA
:100AF000FA01F091FB01309709F00995EF91FF9110
:100B00000895FC018591803011F0EFDFFBCF08954F
:100B1000FF27E0E230E247FF0CC0419597FF09C094
:100B2000EDE26095709580959095611D711D811D18
:100B3000911D27FF02C0219530E350E2AA27660FDE
:100B4000771F881F991FAA1FA41710F0A41B639575
:100B50005A95A9F7AA3008F0A95FA05DAF93F39565
:100B6000611571058105910541F7ED3211F4EF939F
:100B7000F395F21718F43F93F395FBCF8F91B5DF00
:100B8000FA95E1F70895E991F9918591803021F086
:100B9000853219F0AADFF9CF089520E0E894559145
:100BA0005532C1F3503311F4689455915A3348F4D7
:100BB000505390F3220F022E220F220F200D250FEB
:100BC000F4CF0EF4219589919991533619F3533747
:100BD00029F1533559F1BC0188279927E8945C36EF
:100BE00021F48991999168945591543639F446EFDE
:100BF0007EF077FF0DC08FEF9FEF0AC055374AE0B8
:100C000039F0583540E121F0523642E009F00895BC
:100C1000FF93EF937DDFEF91FF91B7CFFF93EF93BA
:100C2000FC0181918030B9F360DFFBCFFF93EF933C
:100C300068DFF1CFDF93CF93CDB7DEB72596A3DF83
:100C4000CF91DF91089581E0089581E008950E9499
:100C50002506089508950E942A060895A5E0B0E0AB
:100C6000E4E3F6E00C94332849835A833091FD0184
:100C700089819A81311119C0662399F0222389F064
:100C80000E940F0D182F682F89819A810E94EB0C0A
:100C900069817A81812F0E94A1132596E3E00C944B
:100CA0004F280E94FD0C182FF3CF0E940F0D698171
:100CB0007A81F1CFFC01262F4081518162817381BD
:100CC00084810E942E06089581E00895CF93DF93DA
:100CD000EC0160E00E945A06BE010E942B06DF91E3
:100CE000CF9108950E94C21408950E94C6140895D9
:100CF00008950E943A0B0E9478062FEF84E39CE04F
:100D0000215080409040E1F700C0000008950E940B
:100D100079060E94672008950E9479060E94782033
:100D200008950F931F93CF93DF938C0161E00E948E
:100D30005A06EC01B8010E942706811106C080E026
:100D4000DF91CF911F910F910895B801CE010E94BC
:100D5000301E8823A1F3B801CE010E9453198823C5
:100D600071F3B801CE010E94A21D882341F3F8015E
:100D700082818823D9F0CB35FDE5DF07A9F170F436
:100D8000C130ECE5DE07B1F0CF3DFCE5DF0721F136
:100D9000C115DC4559F40E948706D1CFCD35EDE56C
:100DA000DE07F9F020F1C83ADD45C1F0C8010E9424
:100DB0002306C6CF90919602892F8E7F90FF816087
:100DC0008093960280FF05C08AEE91E00E94810523
:100DD000B6CF88ED91E0FACF0E94E1110E948C0617
:100DE000AECF0E942211E2CF0E942C11DFCF0E94D1
:100DF0003011DCCF0E94981F0E943C0708950E948A
:100E000040070E949D1F0895829590E09C01220F4B
:100E1000331F220F331F2C7C9595879595958795C9
:100E20008373282B30E0C901880F991F8A7A359582
:100E300027952575822B0895CF93DF93D92F0E9494
:100E40000407C82F8D2F0E9404079C2FDF91CF919C
:100E5000089508950E942907089581E008950E9449
:100E60002D0708950895CF93C82F0E942A078C2F2D
:100E70000E942F07CF91089580E00E9433070895C4
:100E80000E948C1E0E9433070895CF930E948C1EEF
:100E9000C82F8091FC018C1739F1C093FC0180911F
:100EA000960282FF1EC080FF1CC082E092E00E947A
:100EB00081058091960280FF14C01F92CF938DEF21
:100EC00091E09F938F930E941A06809196020F9053
:100ED0000F900F900F9080FF04C08BEF91E00E9465
:100EE00081058C2F0E943307CF910895ABE0B0E0CD
:100EF000ECE7F7E00C9434284F83588769877A87AA
:100F00008B8761110E945A101E821D8285E0FE01AE
:100F10003796DE01119601900D928A95E1F78C814A
:100F20009D81892B61F449815A816B817C818D81FE
:100F30009E810E94830F2B96E2E00C9450288981B9
:100F40009A8189238F3F79F3CE0101960E9464062E
:100F50008111E9CFF0CFFC01808191810E94490D80
:100F60000895CF93C82F8823C9F08238C9F40E940E
:100F70008C1E81FD13C089E30E9412100E947B1019
:100F80002FEF81EE94E0215080409040E1F700C0C7
:100F9000000089E30E941A100E947B10CF910895EF
:100FA0008338A1F40E948C1E80FDF8CF83E50E9457
:100FB00012100E947B102FEF81EE94E021508040B0
:100FC0009040E1F700C0000083E5E4CF8438A1F44D
:100FD0000E948C1E82FDE2CF87E40E9412100E94C4
:100FE0007B102FEF81EE94E0215080409040E1F79C
:100FF00000C0000087E4CECF8CEF8C0F813AB8F4AC
:101000008C2F0E944E1D8111C9CF6C2F8091000141
:10101000909101010E94291F882329F08C2F0E94A2
:101020001A100E947B108C2F0E941210B5CF80E204
:101030008C0F883048F4C77081E001C0880FCA95D2
:10104000EAF70E943D10A8CFEBE5EC0FE33040F447
:10105000F0E0EB5BFE4F808190E00E94EB1E9ECFA4
:10106000E8E5EC0FE73150F4F0E0EE0FFF1FE95E2A
:10107000FE4F808191810E94011F90CFCD3E08F4E8
:101080008DCF8C2F0E94DF160E94B21787CF882346
:1010900009F455C0823879F40E948C1E81FF4FC03C
:1010A00089E30E9412100E947B1089E30E941A10AB
:1010B0000E947B100895833859F40E948C1E80FF93
:1010C0003EC083E50E9412100E947B1083E5EECFA4
:1010D000843859F40E948C1E82FF31C087E40E943C
:1010E00012100E947B1087E4E1CF9CEF980F913A99
:1010F000E8F290E2980F983050F4877091E001C0C8
:10110000990F8A95EAF7892F0E944310D1CF9BE56A
:10111000980F933028F490E080E00E94EB1E089531
:1011200098E5980F973128F490E080E00E94011F25
:1011300008958D3E20F00E9439170E94B21708953D
:101140001F93CF93DF93182FEB010E94B1072097D5
:1011500039F4812F0E944708DF91CF911F910895A4
:101160008FE99FE00197F1F700C000002197EFCFD2
:1011700070E060E0893311F460E570E00E94A0083F
:101180000895882321F00E943D100E947B1008954D
:10119000882321F00E9443100E947B100895B0E044
:1011A000A0E0E5EDF8E00C942D286C01D62FC72FB8
:1011B000FC011281F580F2949FE0F9220E94331025
:1011C000E82E8823B9F0E12E1123A1F08C2F807F27
:1011D000803421F080E28D0F8830D0F08091CA02F7
:1011E00082FF16C082E00E94DE100E94331091E060
:1011F000E82EE926BC2EB2948FE0B822FBE0FB1566
:1012000008F468C0EB2DF0E0E054F74D0C941E2874
:10121000E12CF0CF0C2F0F70C07F11F00295007FF2
:10122000112399F0002359F080E28D0F883010F0DF
:10123000D11107C0802F0E943D100E947B108D2F7E
:1012400041C0802F0E944D10F8CF8D2F0E9447087B
:10125000002309F43FC080E28D0F883010F0D111D7
:1012600004C0802F0E94431003C0802F0E9453109F
:101270000E947B102FC00C2F0F70C07FC03211F066
:101280000295007FDD2381F0D13009F463C0112382
:1012900009F46DC0FF2009F463C0F601858180FF69
:1012A000CECF8F7085835CC08091CA0282FD33C02F
:1012B000112359F0002329F0802F0E943D100E9435
:1012C0007B1080E00E94B10705C080E00E944708C3
:1012D0000111C7CFEB2DE850FF0B349720F40E948B
:1012E0008C1E0E943307EE2089F00E942F1080FD93
:1012F0000DC0F60112820E9429100E94F30BC60154
:101300000E94FA0A0E9429100E94150CCDB7DEB780
:10131000E9E00C944928112389F0F11006C00E94DD
:101320005D10802B0E94C108D5CF21E0F212F7CFCB
:101330000E945D10802B0E946410CCCFF11006C07B
:101340000E947110802F0E94C808C4CF31E0F316AC
:1013500009F2F6CF112331F085E08F1508F4BACFEA
:10136000802FE0CF94E09F1508F4B4CFEBCFFF209F
:1013700049F3D93349F4FFEF27EE33E0F150204031
:101380003040E1F700C000008D2F0E944708A2CF37
:101390008C2F86958695837069F0813009F09ACFFD
:1013A0008D2F9C2F9370111102C090E080E00E945D
:1013B000011F90CF8D2F9C2F9370111102C090E0D0
:1013C00080E00E94EB1E86CF8D2F112329F00E9412
:1013D000DF160E94B2177ECF0E943917FACF8C2FEA
:1013E000837009F041C0111175CF4D2F429546957C
:1013F0004770440F440F0D2F0F7010E030E020E0D5
:10140000042E04C0000F111F221F331F0A94D2F7AD
:1014100060E070E0CB01D4FF0FC06FE070E080E0CF
:1014200090E004C0660F771F881F991F4A95D2F776
:101430006095709580959095C695C695C370602B04
:10144000712B822B932BC23049F058F4C13019F024
:101450000E949E0B3FCF0E948B0B3CCF0E94B10B92
:1014600039CF0E94880B36CF8695112311F08C2F2F
:101470008170882309F42ECF4D2F429546954770F1
:10148000440F440F0D2F0F7010E030E020E0042EC9
:1014900004C0000F111F221F331F0A94D2F760E00F
:1014A00070E0CB01D4FF0FC06FE070E080E090E00F
:1014B00004C0660F771F881F991F4A95D2F7609561
:1014C000709580959095C695C695C370602B712BCD
:1014D000822B932BC23049F058F4C13019F00E948E
:1014E0006E0CF8CE0E945B0CF5CE0E94810CF2CE01
:1014F0000E94CA0BEFCECF70112329F08C2F0E94CF
:10150000F30B8D2F0FCF8D2F0E94C8088C2F0E94B8
:10151000150CE0CED23F51F160F4D03FB9F0D13F8D
:1015200081F0112309F449C0F11089CE8C2F8F71FD
:1015300021C0D33F11F1D43FA1F78091CA0282FDAF
:1015400026C08C2F8F71112311F314C0112349F081
:1015500084E08F1508F4BECE8C2F8F710E94390C59
:10156000B9CE95E09F1508F4B5CEF6CF8C2F8F71CC
:101570001111CDCF0E94F30BADCE112329F08C2F8A
:101580008F710E94DD0BA6CE0E94D70BA3CE112334
:1015900049F0CF718C2F0E94F30B63E08C2F0E94D7
:1015A000C01098CE81E00E94DE10E1E0EF1508F057
:1015B00091CE82E00E94DE108DCEF110DACE8C2F1B
:1015C0008F71A5CF0F931F93CF93DF93EC016881A9
:1015D00079818A810E94540D8C010E94940C0E9492
:1015E000870BB801CE010E94CF08DF91CF911F91E8
:1015F0000F910895CF93DF93EC018B819C81892B10
:1016000029F08881998189238F3F51F4DF91CF910F
:101610000895CE010E94E20ACE010E946606F6CF2E
:10162000CE010E9491068111F4CF0E9433108823CD
:1016300069F38A81882351F38091CA0282FFE6CF41
:1016400082E00E94DE10E2CF90E080E00E94EB1E7C
:1016500090E080E00E94011F0E945A100E947B10BF
:101660000E9445190E94B21708950E9422100E94FC
:10167000240B08950E944A100E94350B08959295FC
:101680009F70963091F058F4925F9F70923058F4AA
:10169000803F19F030F4883E30F481E008959A5F7D
:1016A000F4CF843FD1F380E00895883EB0F3813FCA
:1016B000D1F7F3CFFC01808191810E94490D0E94F6
:1016C0003F0B0895A5E0B0E0E8E6FBE00C94342879
:1016D0002596E2E00C945028A6E0B0E0E2E7FBE0BB
:1016E0000C9434282696E2E00C94502808950E9429
:1016F000760B08950E94770B609334027093350245
:1017000080933602909337020E94240B0895089527
:101710000E947A0B08950F931F9300913402109149
:1017200035022091360230913702602B712B822BCB
:10173000932B0E947A0B1F910F9108950F931F9383
:101740000091340210913502209136023091370217
:1017500060237123822393230E947A0B1F910F91A0
:1017600008950F931F930091340210913502209138
:1017700036023091370260277127822793270E9413
:101780007A0B1F910F9108950E94760B08950E9485
:10179000C40B08950E94C70B60933002709331020E
:1017A00080933202909333020E94240B089560E0EC
:1017B00070E0CB010E94CA0B08950F931F9341E084
:1017C00050E060E070E08A019B0104C0000F111F2F
:1017D000221F331F8A95D2F7C901B8010E94CA0B94
:1017E0001F910F9108950F931F9341E050E060E027
:1017F00070E004C0440F551F661F771F8A95D2F70B
:101800008091300290913102A0913202B091330266
:101810008A019B01082B192B2A2B3B2BC901B801EC
:101820000E94CA0B1F910F9108950F931F9341E0DF
:1018300050E060E070E004C0440F551F661F771F42
:101840008A95D2F7CB01BA016095709580959095F5
:101850000091300210913102209132023091330216
:1018600060237123822393230E94CA0B1F910F913F
:1018700008950F931F9341E050E060E070E004C0D2
:10188000440F551F661F771F8A95D2F7809130024B
:1018900090913102A0913202B09133028A019B01F2
:1018A000082719272A273B27C901B8010E94CA0B1C
:1018B0001F910F9108950F931F9300913002109183
:1018C00031022091320230913302602B712B822B36
:1018D000932B0E94CA0B1F910F9108950F931F9392
:1018E0000091300210913102209132023091330286
:1018F00060237123822393230E94CA0B1F910F91AF
:1019000008950F931F93009130021091310220919E
:1019100032023091330260277127822793270E9479
:10192000CA0B1F910F9108950895262F277091E0FB
:1019300001C0990F2A95EAF723E0769567952A95D5
:10194000E1F725E0269FF001279FF00D1124E40F19
:10195000F51F50E040E0682F70E08191DF011197A2
:101960009B01042E02C0369527950A94E2F7217058
:1019700021952827292328272C934F5F5F4F453037
:10198000510559F70895A82FA77023E096958795DC
:101990002A95E1F725E0289FF001299FF00D1124F9
:1019A000E60FF71F50E040E080E0219130E00A2E82
:1019B00002C0369527950A94E2F721703327042E4A
:1019C00001C0220F0A94EAF7822B4F5F5F4F453028
:1019D000510559F70895262F953070F48F3060F433
:1019E000682F70E08FE0989F600D711D11244EEFFD
:1019F00051E0822F0E94950C0895292F953068F4AC
:101A00008F3058F490E06EEF71E03FE0239F800D3F
:101A1000911D11240E94C30C089580E00895B0E048
:101A2000A0E0E5E1FDE00C942D288C01C09030028F
:101A3000D0903102E0903202F09033028091340273
:101A400090913502A0913602B0913702C82AD92A66
:101A5000EA2AFB2ACFE1D0E0BC2ED701C6010C2E2A
:101A600004C0B695A795979587950A94D2F780FDFF
:101A700009C0219788F7B12C8B2DCDB7DEB7E9E0EF
:101A80000C944928B8018C2F0E94BC13019789F34C
:101A9000F3CFCF93DF93EC010E940F0DBE010E94A4
:101AA000BC13DF91CF9108951F93CF93DF93EB0188
:101AB0009091FD01992339F0CB010E94490DDF91EE
:101AC000CF911F910895882369F0CB010E940F0DDB
:101AD000182F682FCE010E94EB0CBE01812F0E94AF
:101AE000BC13EDCFCB010E94FD0C182FF6CF1F9336
:101AF000CF93DF93C091380216E0809139028C13A6
:101B000004C0DF91CF911F910895D0E01C9FF00198
:101B10001D9FF00D1124E65CFD4F408151816281D3
:101B20007381848195810E946C0B2196C770E5CFEB
:101B300040916A0250916B0260916C0270916D024B
:101B400080916E0290916F020E946C0B08951F931A
:101B5000CF93DF9380916F02807F09F049C080911D
:101B60006C02882309F444C080913802C091390284
:101B700060916A0270916B02A0916D02B0916E0249
:101B8000D62FD72316E0C81799F190E0109711F0DF
:101B9000DF3F19F401968770F6CF189F9001199FC7
:101BA000300D1124F901E65CFD4F41814713F2CF5E
:101BB00040814613EFCF42814111ECCF43815481E4
:101BC0004A1B5B0B483C510528F780916F028F70D0
:101BD000806180936F02F901E15CFD4F80818F701D
:101BE000806180838AE692E00E94FA0A0E94770D63
:101BF000DF91CF911F910895A1E1B0E0E2E0FEE016
:101C00000C942C288C0185E0F801DE011D960190D2
:101C10000D928A95E1F7F801E2808AE6C82E82E00B
:101C2000D82E60916D0270916E026115710509F4F4
:101C30004EC190916A0220916B02892F82238F3FBF
:101C400009F445C140815181A380B480F0906C02B9
:101C5000F501E61BF70BFF2009F4EAC080916F0243
:101C6000382F307FE83CF10508F0A3C031116DC07A
:101C7000FE2C251316C0941314C0E11012C08F70EF
:101C8000806180936F020E94980DC6010E94FA0A3B
:101C900080916F02F80185838F2D6196EAE00C94A4
:101CA0004828A114B10429F0842F85238F3F09F01F
:101CB00027C180E0F82FF170DF2E80FF3CC08091BB
:101CC00038022091390236E0821315C04D875E87B5
:101CD0008D859E850E94490D292F22952F702230D7
:101CE000F0F0243018F59F70F1F0F8019581907FA5
:101CF000D1F4D12C1EC090E0389FF001399FF00D37
:101D00001124E65CFD4F6181651306C06081641398
:101D100003C06281E6120FC001968770D5CF9F7015
:101D200011F0882331F3805E883018F3C8010E94D7
:101D3000FA0AFD2CB1CFEE2009F4AECF80916F02EC
:101D4000816080936F02F12CA7CF251306C09413F6
:101D500004C0F801EE2009F487C0C8010E945A0BA4
:101D6000882319F1EE2009F180916F02803270F022
:101D700020916A0230916B0238872F831986BB86C7
:101D8000AA868C87CE0107960E94FA0A86E0F8019F
:101D9000AAE6B2E001900D928A95E1F70E94A70DA4
:101DA0000E94980DFF24F39477CFC8010E94FA0A8D
:101DB000F9CF311113C07A2DB98AA88A6E2D89897D
:101DC0000E94620B8AE692E00E94FA0A86E0F6011F
:101DD00011928A95E9F70E94980DB5CF25130FC08F
:101DE00094130DC0E1100BC0F8018583C8010E9457
:101DF000FA0A86E0F60111928A95E9F74DCFC801FB
:101E00000E945A0B882389F2EE2079F280916F02AA
:101E1000803208F4BBCF20916A0230916B023A8382
:101E200029831B82BD82AC828E83CE010196ACCF0A
:101E3000E83CF10508F03EC0FE2CEE2009F4B5CFD9
:101E400025132AC0941328C080916F0280FD1BC007
:101E5000982F907FC1F0F8018583903F31F0982F43
:101E6000907F905F8F70892B8583C8010E94FA0A4A
:101E700086E0F801AAE6B2E001900D928A95E1F7BA
:101E80000E94980D09CF86E0F801AAE6B2E0019021
:101E90000D928A95E1F700CFC8010E945A0B81117B
:101EA00075CF80916F02816080936F02C8010E949C
:101EB000FA0AF2CE7A2DB98AA88A6E2D89890E94F3
:101EC000620B86E0F60111928A95E9F7D9CFEE20F0
:101ED00009F46BCFC8010E945A0BF82E882309F42D
:101EE00064CF86E0F801AAE6B2E001900D928A95EF
:101EF000E1F78AE692E00E94AB070E94A70DC0CFEF
:101F000081E08E25D7CEACE0B0E0E9E8FFE00C94AC
:101F100033284F83588769877A878B879C87CE01C0
:101F200007960E94FC0D882369F08A859B85892B82
:101F300039F04F815885842F85238F3F09F06BC07E
:101F400016E05FC086E0FE013796DE011196019033
:101F50000D928A95E1F78A859B85892B89F388857F
:101F60009F8189238F3F61F32091390230E0C901BD
:101F7000019687709927409138024817190671F425
:101F80000E943A0B109239021092380286E0EAE67B
:101F9000F2E0DF011D928A95E9F7D2CF96E0929F99
:101FA000D001939FB00D1124A65CBD4FFE01319668
:101FB00001900D929A95E1F7809339020E94770D76
:101FC000BFCF819FC0011124865C9D4F0E94FC0DF4
:101FD0008823E9F0E09138021E9FF0011124E65CAD
:101FE000FD4F4081518162817381848195810E947E
:101FF0006C0B8091380290E001968770992780934E
:10200000380280913802909139028913DACF2C96E8
:10201000E3E00C944F2869857A858B859C850E9426
:102020006C0B8ECF682F80910001909101010E946E
:102030005F1F0895682F80910001909101010E9417
:10204000621F089580910001909101010E94651F17
:10205000089580917802859585958595089580915C
:1020600078028770089590917802977081E009F462
:1020700080E0089580918302089590918302892BD6
:102080008093830208958095909183029823909382
:102090008302089510928302089590918202892B01
:1020A0008093820208958095909182029823909364
:1020B0008202089510928202089580917902089513
:1020C00008950E94601008959091CA0292FF08C07E
:1020D00090917902981721F0809379020E94611003
:1020E000089580917902882329F01092790280E086
:1020F0000E9461100895CF93DF93E0910001F09169
:102100000101809183028083E0910001F09101013F
:10211000808190918202892B80839091790299230A
:1021200081F0E0910001F09101018081892B808391
:1021300080910001909101010E94171F81110E945E
:102140007110C0910001D091010148E050E060E7BA
:1021500072E0CE010E946F28892B59F088E0FE01C1
:10216000A0E7B2E001900D928A95E1F7CE010E94BE
:10217000991EDF91CF91089508950E94BC10089593
:102180009091CA0292FF11C098E0899F900111249A
:10219000622B609378020E94F30B80917802859500
:1021A000859585950E94BD1008950E94F30B0895B2
:1021B0001092780280E00E94BD10089590917802FC
:1021C0008095892380937802282F277091F4282FF7
:1021D000082E000C330B9217130659F09091CA0287
:1021E00092FF07C08595859585950E94150C0E94E4
:1021F000D8100895CF93C82F8091CA0282FB9927E7
:1022000090F99C17E9F0C0FB82F98093CA02809193
:10221000C9029091CA020E94571182E00E94DE100A
:102220008091960280FF0CC01F92CF938DE092E0C8
:102230009F938F930E941A060F900F900F900F900C
:10224000CF9108958091CA0282FB882780F991E09E
:1022500089270E94FA10089581E00E94FA100895DB
:1022600080E00E94FA10089590E080E00E948428A7
:1022700021E0883E9E4F09F020E0822F089582E001
:1022800090E00E947C28089583E090E00E947C28E2
:102290000895CF9384E090E00E947C28C82F82E2CA
:1022A00090E00E947C28982F8C2FCF910895CF9397
:1022B000C92F682F84E090E00E948A286C2F82E268
:1022C00090E00E948A28CF910895AB01BC018FE075
:1022D00090E00E949C280895AB01BC0183E190E04E
:1022E0000E949C28089560E070E0CB010E946C1170
:1022F000089560E070E0CB010E9465110E947311A7
:10230000089568EE7EEF90E080E00E94A82860E0EB
:1023100082E090E00E948A2860E083E090E00E94E2
:102320008A281092340210923502109236021092CE
:10233000370260E084E090E00E948A2864E082E254
:1023400090E00E948A2860E085E090E00E948A2860
:1023500060E086E090E00E948A286FEF87E090E0DE
:102360000E948A2840E050E0BA0188E090E00E9494
:102370009C2860E08DE090E00E948A2840E050E0D8
:10238000BA0188E190E00E949C2860E087E190E03B
:102390000E948A2840E050E0BA018CE190E00E945F
:1023A0009C2870E060E080E290E00E94A82840E075
:1023B00050E0BA0188E190E00E949C280E947911C7
:1023C00008950E9481110895682F8EE090E00E9488
:1023D0008A2808950E9428206093920270939302A5
:1023E000809394029093950260938E0270938F0273
:1023F00080939002909391020895089508950E9409
:10240000FE11089508950E94021208958BE592E24C
:102410000E94821E0E94FD110E94FF11089581E01A
:1024200008950E940F120895089508950E941412AD
:102430000E94151208950E949C140E94320708956C
:102440000E9413200E94C2150E941B120E940312B8
:102450000895AAE0B0E0EFE2F2E10C9427280E9490
:10246000D815A82E81110E94EA1134E8832E32E09B
:10247000932E10E000E0502E802F0E94C9146C01B2
:10248000F401619071904F016816790609F443C018
:102490008091960281FD0E94D214B12CEE24E39427
:1024A000F12C6C247D24C3018E219F21892B69F19D
:1024B0000E9411128823B1F0BE825F82CE20DF20FD
:1024C00081E0C114D10409F480E088870E941C20B7
:1024D0008160782F9A8789874E815F8168858A8598
:1024E0000E947607000F111FF801EC57FD4F808105
:1024F0009181E826F926F182E08281E0A11001C0F5
:1025000080E02A96EFE00C944328B394EE0CFF1C75
:10251000FFE0BF12C8CF0F5F1F4F0530110509F054
:10252000AACF8FEF89838A831B820E941C2081603F
:10253000782F9D838C8349815A816B818D810E9484
:102540007607DBCF0E9429120E9450180E9445078F
:102550000895CF93DF930E94C113EC01811521E50B
:10256000920708F042C0811530E5930708F09DC03E
:10257000883E910530F5803E910508F092C0883A7A
:10258000910588F4853A910508F084C08130910561
:1025900009F487C0009709F484C0049708F081C04B
:1025A000D0E0C0E07EC08F3B9105D0F7C85AD0E0A4
:1025B000CC0FDD1FC85BDE4F0990D881C02DD464DD
:1025C00070C08115904250F4C11581E0D80708F021
:1025D00068C0CD3ED10520F3D06563C0C11590E43D
:1025E000D907F0F2DF70D06A5CC0811525E592074B
:1025F00000F5811534E5930708F08BC0811543E59C
:10260000940708F073C0C11582E5D80708F469C0C3
:10261000CE018370992721E030E002C0220F331FE2
:102620008A95E2F7C695C69580E2C89FE00111241D
:1026300054C0C11599E5D907A8F4C11528E5D207FA
:1026400008F06CC0C11536E5D30708F0A9CF8C2F70
:102650000E945814C82FD0E0DC2FCC27CC27DF7184
:10266000D0621FC0C1154AE5D40708F45CC0CE0192
:1026700090568115904208F093CF8D2F8F710E9454
:10268000581490E0982F882788279F719C012C2B45
:10269000E901E6CFC55AD0E0CA58DE4FC881D0E084
:1026A000D064CE01DF91CF910895E4E096958795AF
:1026B000EA95E1F783702C2F26952695237040E24A
:1026C000249F90011124382B8C2F8370C1E0D0E01F
:1026D00002C0CC0FDD1F8A95E2F7C22BD32BDC683A
:1026E000E0CFDC2FCC27C16FD06ADBCF8370992776
:1026F00021E030E002C0220F331F8A95E2F7C69531
:10270000C69590E2C99FE0011124C22BD32BDA6851
:10271000C8CFD82FCC27C46FD06AC3CFDC2FCC272B
:10272000C06FD06ABECF8C2F8F700E94581434E0D7
:10273000D695C7953A95E1F7CF709C2FEC01D069FB
:10274000B0CF972F7530A8F46F3098F470E02FE079
:10275000929F600D711D1124FB019BE4899FE00D88
:10276000F11D1124EE0FFF1FE455FF4F8591949149
:10277000089580E090E008950E94A1130E94A9129C
:10278000089582389105B1F1B0F48133910509F4CF
:1027900075C048F48932910509F469C08A329105FF
:1027A00009F473C008958533910509F459C089333C
:1027B000910501F10895833E9105A9F138F4803E19
:1027C0009105F9F0823E910549F10895863E910503
:1027D000A9F1873E9105C9F1843E910519F5209133
:1027E000CA0221FF1FC08091C90284FD14C087EE78
:1027F00090E008952091C9022370A1F080EE90E04E
:1028000008952091C90220FD47C03091CA0230FFCF
:1028100009C024FF44C090E080E004C02091C902B8
:1028200022FDF7CF08952091C90222FD3BC03091CF
:10283000CA0230FDE3CF24FFF5CFEDCF2091C902CE
:1028400023FFF0CF24FDE7CFD2CF2091C90223FD93
:102850002CC03091CA0231FFEECF84EE90E0089593
:102860002091C90225FFDECF89E290E008952091F2
:10287000C90225FFD7CF85E390E008952091C902D2
:1028800026FFD0CF8AE290E008952091C90226FF6A
:10289000C9CF81E390E0089589E390E0089583EE45
:1028A00090E0089582EE90E0089586EE90E008951D
:1028B0009091C90292FF06C0282F28712830F9F4A0
:1028C000877F846093FF06C0282F28712831F1F498
:1028D000877E84612091CA0220FF06C0382F38719C
:1028E0003830D9F4877F816021FF06C0282F2871F6
:1028F0002831D1F4877E816194FD877E0895282F49
:1029000024712430F9F68B7F8860DCCF282F247166
:10291000243101F78B7E8861DDCF382F3171313062
:1029200019F78E7F8860E0CF282F2171213121F7A0
:102930008E7E8861E1CF08950E943411811102C01A
:102940000E94E1110E943F11809396020E9449115A
:102950009093CA028093C9020E949B140E94441162
:10296000682F70E090E080E00E94880B6091300258
:102970007091310280913202909133020E94C70B14
:10298000089508950E94C114089508950E94C514E1
:102990000895E82FF0E0EE0FFF1FEB52FD4F80810E
:1029A00091810895B0E0A0E0E8EDF4E10C942E28C8
:1029B00082E392E00E94810585EDE82E82E0F82E08
:1029C000D0E0C0E09DE2C92E92E0D92E04E212E0F0
:1029D000DF93CF93DF92CF920E941A068AE292E0B1
:1029E0000E948105F701819191917F010E941C074E
:1029F0009F938F931F930F930E941A0682E292E097
:102A00000E94810521968DB79EB708960FB6F8945F
:102A10009EBF0FBE8DBFC530D105D1F6CDB7DEB795
:102A2000E8E00C944A2880EA8A95F1F7089500C0FE
:102A300008950E9413150895F894E82FE295EF7019
:102A4000F0E031A1282F2F7081E090E001C0880FC5
:102A50002A95EAF7982F9095932391A392A1892B19
:102A600082A3789408950F931F93CF93DF93C8E8C0
:102A7000D1E089918F3F11F00E941C1581E0CD3883
:102A8000D807B9F7C9E7D1E008E811E089918F3F8D
:102A900011F00E941C150C171D07C1F7DF91CF9193
:102AA0001F910F910895AF92BF92DF92EF92FF9224
:102AB0000F931F93CF93DF938C01D62EC62FD0E0B8
:102AC000CE0188579E4F7C01FC0120812F3F09F4E5
:102AD0004CC0F894E22FE295EF70F0E031A12F7036
:102AE00081E090E001C0880F2A95EAF7932F982B98
:102AF00091A392A18095892382A378940E941715AF
:102B0000E9E7F1E041E050E0B12CA12C21912F3F09
:102B1000B1F1A22FA295AF70B0E090968C9190E0A9
:102B20002F7002C0959587952A95E2F780FD27C002
:102B3000CA01A82AB92A440F551F81E0E838F807CE
:102B400029F7F70180818F3F11F00E941C1561E089
:102B5000A114B10409F460E08D2D0E941915CC0F69
:102B6000DD1FC00FD11FB982A882DF91CF911F91C5
:102B70000F91FF90EF90DF90BF90AF90089590E09D
:102B800080E0D7CF0E9433158AE0E5EDF2E0DF0167
:102B9000982F1D929A95E9F7EBECF2E0DF011D9278
:102BA0008A95E9F785E00E9414160E94720608953E
:102BB000AAE0B0E0EEEDF5E10C9431288E010F5F54
:102BC0001F4F8AE0F80111928A95E9F7F12C6F2DD9
:102BD000C8010E945315F394F5E0FF12F8CF4AE0C4
:102BE00050E0B8018BEC92E00E946F28FF24F39430
:102BF000009709F4F12C892B41F08AE0F801ABEC45
:102C0000B2E001900D928A95E1F72F2D45E065ED38
:102C100072E08BEC92E00E9415160E9475068F2DD3
:102C20002A96E5E00C944D280895FF920F931F9388
:102C3000CF93DF93F82E092F162FD72FC42F2223DF
:102C400049F081E0809399020E941C2090939802A1
:102C500080939702809199028823A1F08091970236
:102C6000909198020E943420059760F0EF2DF02F8C
:102C7000A12FBD2F90E080E0D0E08C179D073CF0A5
:102C800010929902CDB7DEB7E5E00C944D28219162
:102C900031912D933D930196F0CF0E94D7220E944F
:102CA00020120E94E42208950E94E9220E94A212AA
:102CB0000E94072308950E94B51F0E94BD220E9412
:102CC00006120E944D160E9454160E941612FBCF47
:102CD0008091A00280FF0DC06091070170E0660F37
:102CE000771F6038710570F56115710569F1862FE0
:102CF000089581FF07C06091070184E0689FB001DB
:102D00001124EFCF6091070182FD0AC080919F02DC
:102D10008823A9F02091060160910701821710F025
:102D200088E0ECCF869FC001112433E0880F991F03
:102D30003A95E1F7622F70E00E940A28D2CF68E04E
:102D400070E0D5CF8FE7089581E008958091A002CB
:102D500080FF0CC06091030170E0759567957595D3
:102D600067956115710549F1862F089581FF06C0A9
:102D70006091030170E075956795F3CF6091030151
:102D800082FD0BC090919E029923A1F060910201F7
:102D900080910301961738F0682F70E06038710554
:102DA00000F38FE70895899FC001112470E00E940D
:102DB0000A28F4CF61E070E0D7CF81E008958D3E1E
:102DC00031F40E94681681958093A40208958E3E86
:102DD00019F40E946816F8CF8F3E31F40E946816ED
:102DE00081958093A3020895803F19F40E9468168C
:102DF000F8CF893F29F40E94A6168093A502089572
:102E00008A3F21F40E94A6168195F7CF8B3F31F4BB
:102E10000E94A61681958093A60208958C3F19F40E
:102E20000E94A616F8CF9FE0980F983070F4815F4B
:102E3000990B21E030E001C0220F8A95EAF78091DA
:102E4000A202822B8093A20208958D3F31F48091DB
:102E5000A00281608093A00208958E3F21F48091AA
:102E6000A0028260F7CF8F3FB9F78091A002846003
:102E7000F1CF4091A3028D3E59F48091A40287FFC7
:102E80000DC01092A40241110BC010929F0208C005
:102E90008E3E81F48091A40218169CF3442381F0A5
:102EA0008091A5029091A602892B09F05AC0109238
:102EB0009E0208958F3E49F447FFF0CF1092A3027F
:102EC0008091A4028111ECCFE0CF803F19F4141659
:102ED000ACF3E4CF9091A502893F29F41916F4F6DA
:102EE0001092A502DBCF8A3F19F497FFD7CFF8CF16
:102EF0009091A6028B3F29F497FFD0CF1092A602A3
:102F0000CDCF8C3F19F41916CCF3C8CF9FE0980FA2
:102F1000983090F4815F990B21E030E0B90102C054
:102F2000660F771F8A95E2F7CB0180959091A202F8
:102F300089238093A202B2CF8D3F31F48091A00209
:102F40008E7F8093A002AACF8E3F21F48091A002B1
:102F50008D7FF7CF8F3F09F0A1CF8091A0028B7FAB
:102F6000F0CF08958091960283FF7EC080E792E0C3
:102F70000E9481058091A2021F928F938BE692E0BE
:102F80009F938F930E941A0689E692E00E94810522
:102F90008091A302282F082E000C330B3F938F93B0
:102FA00086E692E09F938F930E941A0684E692E051
:102FB0000E9481058091A402282F082E000C330B5B
:102FC0003F938F9381E692E09F938F930E941A061E
:102FD0008FE592E00E9481058091A502282F082E9E
:102FE000000C330B3F938F938CE592E09F938F936C
:102FF0000E941A068AE592E00E9481058091A6024D
:10300000282F082E000C330B3F938F9387E592E017
:103010009F938F930E941A0684E592E00E94810597
:1030200080919F021F928F9381E592E09F938F93EF
:103030000E941A068FE492E00E9481058091A0020E
:103040001F928F938CE492E09F938F930E941A06B5
:1030500089E492E00E9481058DB79EB74C960FB629
:10306000F8949EBF0FBE8DBF0E941C209C019091C2
:10307000A3028091A402982B21F030939D0220930B
:103080009C029091A5028091A602982B21F030938A
:103090009B0220939A0281EA92E00E94DD1E08952D
:1030A000A6E0B0E0E6E5F8E10C94332886E0E1EA3A
:1030B000F2E0DE01119601900D928A95E1F71092EF
:1030C000A3021092A4021092A5021092A6028B8174
:1030D0009C81892B81F080919C0290919D020E949D
:1030E0003420AC0190919F02992391F180910801C5
:1030F00084171506D0F18D819E81892B91F08091E6
:103100009A0290919B020E943420AC0190919E0201
:10311000992309F46BC0809104018417150608F403
:1031200073C0BE016F5F7F4F81EA92E00E946C1F07
:1031300081110E94B21786E0FE013196A1EAB2E049
:1031400001900D928A95E1F72696E3E00C944F28C2
:10315000209109018AE0289F900111242417350746
:1031600050F69F5F90939F0202C09F3FD1F71B8153
:10317000112359F00E9468169FEF11160CF491E08C
:10318000899F802D11248093A3021C81112359F063
:103190000E9468169FEF11160CF491E0899F802D14
:1031A00011248093A4023091A302332309F4A3CF06
:1031B0002091A402222309F49ECF45EB3403C001E1
:1031C0001124992359F09093A30245EB2403900115
:1031D0001124332339F03093A4028DCF81E0809302
:1031E000A302F3CF81E08093A40285CF2091050153
:1031F0008AE0289F900111242417350708F091CF09
:103200009F5F90939E0202C09F3FD1F71D811123C3
:1032100059F00E94A6169FEF11160CF491E0899FB9
:10322000802D11248093A5021E81112359F00E9444
:10323000A6169FEF11160CF491E0899F802D1124A2
:103240008093A6023091A502332309F46ACF20911E
:10325000A602222309F465CF45EB3403C0011124F3
:10326000992359F09093A50245EB24039001112472
:10327000332339F03093A60254CF81E08093A50226
:10328000F3CF81E08093A6024CCF86E0E1EAF2E042
:10329000DF011D928A95E9F710929F0210929E021B
:1032A0001092A0020895CF93DF93EC01FB0182817D
:1032B000882309F433C1C430FDE5DF07C0F5CB3FF7
:1032C0009CE5D90730F49E0122503C45243131055C
:1032D000B0F50E9449119093CA028093C902C1318E
:1032E0008CE5D80709F4EEC008F069C0C930ECE5F8
:1032F000DE0709F4D5C0C8F5C5308CE5D80709F458
:10330000C7C000F5C330ECE5DE0709F4B9C008F02A
:10331000BBC0C230DC4509F4ADC08091C9029091B8
:10332000CA020E9457110E943A0B80E008C0C236C0
:10333000EDE5DE0771F2C63AFDE5DF0751F2DF91F8
:10334000CF9108958091C9028062C7309CE5D9076A
:1033500009F493C08091C9028061C830DC4508F44B
:103360008CC08091C902806488C08091C9028B7F23
:10337000CD30FCE5DF0709F480C098F48091C902E4
:103380008E7FCB309CE5D90709F477C08091C902C4
:103390008C60CC30DC4508F470C08091C9028D7F10
:1033A0006CC08091C9028F7ECF30FCE5DF0709F445
:1033B00064C008F47BC08091C9028F7D5EC0CE3F9F
:1033C0009CE5D90709F47AC050F5C531FCE5DF0763
:1033D00009F486C098F48091C902837FC3319CE5CB
:1033E000D90709F44AC008F471C00E943A0B9091C1
:1033F000C902892F97FB87F980583FC0CC3FFCE575
:10340000DF0709F449C008F055C08091CA02816005
:10341000CB3FDC4509F081CF8093CA027ECFC2301A
:10342000EDE5DE0709F468C0A8F4C1158DE5D807FD
:1034300009F452C08091CA028360C130DD4560F357
:103440008091CA02982F909591708E7F892B90FB66
:1034500081F9E2CFC236EDE5DE0709F451C0C63A84
:10346000FDE5DF0709F453C0C330DD4509F055CF52
:1034700080E043C08091C90281608093C9024DCF32
:103480008091C9028260F9CF8091C9028460F5CF32
:103490008091C9028860F1CF8091CA028260BCCF5E
:1034A0000E943A0B8091C9028068E7CF8091C902DF
:1034B000877FE3CF8091CA028E7FAECF8091CA0210
:1034C0008D7FAACF8091C9028F7BD7CF0E943A0B04
:1034D0008091C9028F77D1CF8091CA028C7F9CCF17
:1034E0008091C90282FB992790F921E0922790FBF5
:1034F00082F990FB83F9C1CF81E00E94E4110DCFE6
:103500009091C902892F8F7E94FF8061B6CF9091F0
:10351000C902892F8E7F90FF8160AFCF81E00FCFEE
:10352000809102011F928F93809103011F928F93CC
:10353000809106011F928F93809107011F928F93B4
:10354000809108011F928F93809109011F928F93A0
:1035500083E992E09F938F930E941A068DB79EB7DE
:103560000E960FB6F8949EBF0FBE8DBF0895883299
:1035700028F58E3108F072C08B3041F130F487307D
:1035800009F4CFC082EF93E0E0C0833109F45FC05B
:103590008431C1F784E194E00E9481058091AB02FF
:1035A000882309F4FEC01092AB021092AA02109276
:1035B000A9021092A8021092A70220C08F3409F429
:1035C000C7C0D8F5893231F38833E1F687E194E05A
:1035D0000E9481050E94901A1F9281E08F931F9292
:1035E00088E08F9380E193E09F938F930E941A0667
:1035F0000F900F900F900F900F900F902091AB02B3
:10360000222309F4C9C08091A7029091A8020097D3
:1036100011F48DE891E09F938F931F922F9380EE8A
:1036200093E09F938F930E941A060F900F900F9034
:103630000F900F900F9081E00895813509F49CC0A0
:1036400008F49CC0823509F09DCF81E082C086E0FD
:1036500094E00E9481050E94901AD0CF8D518093F2
:10366000AB02833009F442C058F48130C1F082309B
:10367000A1F11092AB0283E094E00E9481051BC08F
:10368000853009F445C0D8F1863099F782E091E0A1
:103690009093AA028093A90285ED91E008C089E089
:1036A00091E09093AA028093A90281E991E090931E
:1036B000A8028093A7028091AB02882309F49ECFD1
:1036C0001F928F938FEF93E09F938F930E941A0620
:1036D0000F900F900F900F9091CF88E091E0909312
:1036E000AA028093A9028AE991E0E1CF87E091E004
:1036F0009093AA028093A90286EA91E0D8CF86E04F
:1037000091E09093AA028093A90283EB91E0CFCF3E
:1037100083E091E09093AA028093A90282EC91E069
:10372000C6CF81E08093090184E1809308018AE09B
:10373000809307018EE18093060188E08093030166
:1037400088E28093020185EF93E00E94810556CFC5
:103750008AE0E091A902F091AA023097D1F020818D
:10376000082E000C990B820F911D8F3F910541F09F
:103770003CF08FEF808307C08FEFEBCF86EFE9CF70
:1037800097FFF8CF108280811F928F938CEE93E089
:103790009BCF89EE93E0D9CF8CED93E00E94810519
:1037A0004ACF80E00895CF93C82F1F928F938DE268
:1037B00094E09F938F930E941A0661E070E080E08E
:1037C00090E004C0660F771F881F991FCA95D2F733
:1037D0000E94880B0E943A0B0F900F900F900F9051
:1037E000CF910895EF92FF920F931F93CF93DF93A2
:1037F0008B3109F4FFC008F09FC08B3009F4BBC0C7
:1038000008F07DC0863009F4C9C048F4853009F459
:10381000A1C08BE698E00E94810580E0CFC0873090
:1038200009F4D1C08830A9F70E9444111F928F93E8
:103830008EE498E09F938F930E941A060E943F1196
:1038400083FB992790F91F929F9382FB992790F908
:103850001F929F9381FB992790F91F929F93982F16
:1038600091701F929F931F928F9385E098E09F9392
:103870008F930E941A060E94491187FB222720F984
:103880001F922F9386FB222720F91F922F9385FBEF
:10389000222720F91F922F9384FB222720F91F92C1
:1038A0002F9383FB222720F91F922F9382FB22273D
:1038B00020F91F922F9391FB222720F91F922F931B
:1038C000292F21701F922F9381FB222720F91F920D
:1038D0002F93282F21701F922F939F938F9380E215
:1038E00097E09F938F930E941A068DB79EB7889694
:1038F0000FB6F8949EBF0FBE8DBF81E05FC08031D0
:1039000009F490C080F48E3009F083CF9091960234
:10391000892F8B7F92FF84608093960282FF7FC005
:1039200086E998E073C0863109F48CC0893109F0CA
:1039300070CF8DE994E021C08A3249F190F487324A
:1039400011F128F48E3108F464CF8D511DC08932F5
:1039500009F05FCF89ED98E00E9481050E948706FB
:10396000CCCF833468F48A3308F091C0853359F0A2
:10397000883309F04ECF8DE795E00E948105BDCFD9
:10398000833409F046CF80E00E94D31BB6CF89EF85
:1039900098E00E9481050E94E111AFCF80919602CC
:1039A000807F8093960286E595E00E94810585EFF1
:1039B00098E00E94810581E08093AC02CDB7DEB72C
:1039C000E6E00C944C2890919602892F8E7F90FF10
:1039D00081608093960280FF03C08DEC98E0CDCF8C
:1039E00080EC98E00E94810580919602817F80930F
:1039F000960283CF90919602892F8D7F91FF8260EE
:103A00008093960281FF08C083EB98E00E948105B5
:103A1000809196028160EBCF85EA98E0AECF86E890
:103A200098E0ABCF90919602892F877F93FF8860B3
:103A30008093960283FF03C08AE798E0E7CF8DE684
:103A400098E09BCF0E942820162F072FF82EE92EF2
:103A5000D091C802C09116010E948C1EEF92FF9275
:103A60000F931F931F92DF931F92CF931F928F93F9
:103A700082E394E09F938F930E941A068DB79EB7BE
:103A80000C960FB6F8949EBF0FBE8DBF36CF8953EC
:103A90007BCF80E008950E94491D0895CF93C82FE1
:103AA0008091AC028130C1F0882339F0823009F472
:103AB00044C01092AC0280E00DC00E943A108232E5
:103AC000D1F78C2F0E94491D81111BC08C2F0E94A1
:103AD000F21B8170CF9108950E943A10823289F3CF
:103AE0008C2F0E944B1D81111BC0C431D9F060F492
:103AF000CB3071F0C031D1F087E294E00E948105B3
:103B000013C081E090E0E5CFC93261F0C833A1F77E
:103B100086E595E00E94810589E294E00E94810596
:103B200081E0D7CF1092AC0280E0D3CF82E08093C7
:103B3000AC0288E30E94B71AF3CF8C2F0E94B71A09
:103B400081E0C8CFCF93DF93EB0186319C4511F51F
:103B50000E943A109A81992399F08A7A91E009F4A7
:103B600090E09093AD02811109C089E20E94121089
:103B70000E947B1080E0DF91CF91089585E3F6CF1E
:103B80008091AD02811104C089E20E941A10F0CF29
:103B900085E3FBCF81E0EFCF0F931F93CF93DF93AC
:103BA000C42FD22FFC0182818823C9F04093B00238
:103BB0000E941C209093AF028093AE0280E28C0F93
:103BC000883040F4C77081E001C0880FCA95EAF7D9
:103BD0000E94C108DF91CF911F910F91089510911C
:103BE000B002141332C08091AE029091AF020E94D5
:103BF0003420883C910548F5C0E2CD0F1D17B9F07F
:103C000080E2810F883040F4177081E001C0880F96
:103C10001A95EAF70E94C808C83048F481E09D2F41
:103C2000977001C0880F9A95EAF70E94C108802F0B
:103C30000E94B808C83070F6D77081E001C0880FC4
:103C4000DA95EAF70E94C808C5CF80E28C0F883069
:103C500008F6C77081E001C0880FCA95EAF7F2CF75
:103C60000F939C01CB01243F4CE5340759F1A8F494
:103C7000293DFCE53F0701F12A3D4CE53407D1F130
:103C8000283D3C4591F406E221EE41EE68ED7CE5ED
:103C90000E94CC1D80E00F910895263FFCE53F0770
:103CA000E9F0B0F0273F3C45F9F0FC018281882320
:103CB00039F11092B002EFCF07E225EE45EE69ED43
:103CC0007CE5E6CF06E221EE40EE64EF7CE5E0CF56
:103CD00007E225EE44EE65EF7CE5DACF06E221EE61
:103CE00042EE66EF7CE5D4CF07E225EE46EE67EFC5
:103CF0007CE5CECF08E221E045EE6AED7CE5C8CF59
:103D000081E0C9CF9093FB018093FA0108959093CD
:103D1000B6028093B5020895E091B502F091B60223
:103D2000309729F00190F081E02D0995089580E009
:103D30000895EF92FF920F931F93CF93DF938C011F
:103D4000E091B502F091B602309791F10280F381D3
:103D5000E02D09958091960282FF2AC080FF04C061
:103D600082E199E00E948105D0E0C0E08CE0E82E7D
:103D700089E0F82E8091960280FF0EC0F801EC0FCA
:103D8000FD1F80811F928F93FF92EF920E941A066F
:103D90000F900F900F900F902196C830D10551F7DA
:103DA0008091960280FF04C08AE099E00E9481051C
:103DB000CDB7DEB7E6E00C944C28E091B502F09167
:103DC000B602309739F022E0DC012C930480F581B3
:103DD000E02D099508952091B3023091B40228177F
:103DE000390771F09093B4028093B302E091B50269
:103DF000F091B602309721F00680F781E02D099509
:103E000008952091B1023091B2022817390771F05C
:103E10009093B2028093B102E091B502F091B602A4
:103E2000309721F00084F185E02D099508959C01DB
:103E30002E5F3F4FAC01485F5F4F80E0241735078E
:103E400009F40895F90191919F019923B9F38F5FC6
:103E5000F5CF662349F0FC0132960896219126178A
:103E600029F0E817F907D1F780E0089581E0089577
:103E70009C01FC0132969FEF80E04191461751F082
:103E80009F3F19F4411101C0982F8F5F8630A9F729
:103E90009F3F09F40895290F311D97FD3A95F901C7
:103EA00062830895FC01329608962191261303C07F
:103EB000DF0111971C92E817F907B9F708950E94DE
:103EC000381F08950E94521F0895029626E0FC01B3
:103ED00011922A95E9F7089546E050E00E946F2874
:103EE00021E0892B09F420E0822F089508950E9493
:103EF000761F0895811106C081E08093B7020E9469
:103F0000771F089582E0F9CF83E08093B7020E9483
:103F1000771F08950E947A1F089581E08093B70269
:103F20000E94771F08950E948D1F08950895089597
:103F30000E94971F0895089508950E94961F08955E
:103F4000CF930E949B1F0E94D8150E949C1FC0E027
:103F50008C2F0E94C914892B31F4CF5FC530C1F773
:103F600080E0CF91089581E0FCCF85B7806885BF60
:103F700085B7806885BF08951F921FB61F921124D0
:103F80008F939F93AF93BF938091B802811113C019
:103F90008091DF029091E002A091E102B091E202F3
:103FA0004196A11DB11D8093DF029093E002A09382
:103FB000E102B093E202BF91AF919F918F911F9068
:103FC0001FBE1F9018958091E702843031F10E9446
:103FD000FA061092B80288E190E020E40FB6F89457
:103FE000A895809360000FBE2093600083B7817F07
:103FF000846083BF83B7816083BF7894889583B7DB
:104000008E7F83BF0FB6F894A89580916000886179
:1040100080936000109260000FBE08950E943A0BDA
:104020000E94FF06089582E084BD93E095BD9AEF5B
:1040300097BD80936E0008952FB7F8948091DF02AA
:104040009091E002A091E102B091E2022FBF0895A9
:104050002FB7F8946091DF027091E0028091E10245
:104060009091E2022FBF08959C014FB7F894809180
:10407000DF029091E002A091E102B091E2024FBF15
:10408000821B930B089578941F921FB61F921124E0
:104090008F939F93AF93BF938091DF029091E00243
:1040A000A091E102B091E2020196A11DB11D8093A1
:1040B000DF029093E002A093E102B093E202BF918D
:1040C000AF919F918F911F901FBE1F90189587E70A
:1040D00097E7909301088093000888E19AE00FB673
:1040E000F894A895809360000FBE90936000FFCF76
:1040F00088E19AE00FB6F894A895809360000FBE0F
:1041000090936000FFCF8091C702089508959C01AD
:1041100082E08093E9009FEF8091E800915085FD57
:1041200006C085ED8A95F1F700009111F5CF8091D9
:10413000E80085FF0CC050E040E066E070E0C90197
:104140000E9478238091E8008E778093E80008959C
:10415000CF93DF93EC0181E08093E9008FEF9091A2
:10416000E800815095FD06C095ED9A95F1F70000A5
:104170008111F5CF8091E80085FF14C050E040E048
:1041800068E070E0CE010E9478238091E8008E778D
:104190008093E80088E0FE01AFEBB2E001900D9261
:1041A0008A95E1F7DF91CF9108958093BB027093D8
:1041B000BD026093BC028091E702843001F582E089
:1041C0008093E9008FEF9091E800815095FD06C043
:1041D00095ED9A95F1F700008111F5CF8091E800F7
:1041E00085FF0DC050E040E063E070E08BEB92E0B3
:1041F0000E9478238091E8008E778093E8000895EC
:10420000BC0184E00E94D5200895BC0183E00E9497
:10421000D520089588E399E00E9481058091E60207
:10422000811109C00E9408250E9465258091E20045
:1042300084608093E200089584E399E00E94810500
:104240001092E602089580E399E00E9481050E94A1
:104250008D1F08958CE299E00E9481056091E30230
:1042600081E0611101C080E00E94841F089588E20E
:1042700099E00E9481059091E70281E0943009F075
:1042800080E06091E3020E948A1F08952091BA02A3
:104290002F5F822F62E30E94FE27992319F020935B
:1042A000BA0208951092BA028091BE028823F1F0FA
:1042B0008091E7028430C1F49091E9009F702091D1
:1042C000EC00822F817020FD80E8892B93E0909391
:1042D000E9009091EB0090FF04C09091EE0097FDF3
:1042E00008C08F708093E9001092BE02089510926A
:1042F000F1009091E80095FDFACF9091E80090FFD1
:10430000F0CF9091E8009E779093E800EACF42E0EA
:1043100061EC81E00E94842442E261EC82E00E9430
:10432000842442E261EC83E00E9484249091E702BD
:1043300081E0943009F080E06091E3020E947A1FEE
:1043400008958091E902833009F461C030F481302E
:10435000D1F1823009F49EC008958A3009F48AC0F0
:104360008B3009F46FC0893009F050C08091E802A9
:10437000813209F04BC08091EC029091ED020297DE
:1043800008F044C08091E800877F8093E800809126
:10439000E80082FF37C09091F3008091F20002970D
:1043A00031F48091F100813011F0863021F4809158
:1043B000F1008093C7028091E8008B778093E8003A
:1043C0000E94B82423C08091E802813AF9F48091D8
:1043D000E800877F8093E8008091EC029091ED02E5
:1043E000892B61F468E08FEB92E070E00E94C723B4
:1043F0008091E8008B778093E800089560E090E07A
:1044000080E0F3CF8091E7028111C1CF08958091C0
:10441000E802813AD9F78091EC029091ED02892B64
:10442000A9F78091E800877F8093E8008091E800F9
:1044300080FFFCCF809116018093F1008091E8000D
:104440008E77BCCF8091E802813201F78091EC0237
:104450009091ED02892BD1F68091E800877F8093BF
:10446000E8000E94B8248091EA02809316010E941D
:104470003A0B08958091E802813241F68091E8007C
:10448000877F8093E8000E94B8248091EB0280939C
:10449000C80208958091E802813A09F0B7CF80916F
:1044A000E800877F8093E8008091E80080FFFCCFE0
:1044B0008091C802C1CF9FB7F8941092BE029FBFEF
:1044C0009091E702943009F048C02091E9002F70E4
:1044D0003091EC00932F917030FD90E8922B23E007
:1044E0002093E9002091EB0020FF34C02091EE00E2
:1044F00027FF30C02091B902222321F02091E8004B
:1045000025FF28C01092B90226E03091E80035FF5F
:1045100014C08093F1008091E80085FD27C0809150
:10452000E80080FFFCCF8091E8008E778093E80060
:104530009F709093E90080E008953091E702343055
:1045400049F43091EB0035FD05C0215041F481E084
:104550008093B9029F709093E9008FEF0895EFE97F
:10456000FFE03197F1F700C00000CFCF8FB7F8948C
:1045700021E02093BE028FBFDBCF84B7877F84BF4B
:104580000FB6F894A89580916000886180936000D0
:10459000109260000FBE80E890E00FB6F894809310
:1045A0006100909361000FBE0E94931F08950E94C6
:1045B00008250E946525E2EEF0E08081846080831A
:1045C00078940E94E32708958AE091E00E94871E74
:1045D00008958091E702853051F484E299E00E94C9
:1045E00081058091E702853019F00E940E20089520
:1045F0000E94E31F8091E502882399F30E94A01F87
:10460000882379F30E9462230E943A0BEACF08952F
:104610000E940B230895292F33272330310521F1E0
:1046200068F42130310509F443C02230310509F422
:1046300044C090E080E030E020E026C02132310527
:1046400051F122323105A9F76330710590F7FB0172
:10465000EE0FFF1FE351FE4F2081318166517E4FE7
:10466000FB01808190E010C099278130910581F095
:10467000009729F00297E9F6ECE3F9E002C0EEE5D5
:10468000F9E0849190E09F01FA013183208308953D
:10469000ECE4F9E0F6CF6330710558F6660F771F4A
:1046A000FB01ED50FE4F2081318189E090E0ECCF9D
:1046B00082E190E02DEB39E0E7CF8BE590E022E658
:1046C00039E0E2CF80E189BD82E189BD09B400FE15
:1046D000FDCF8091D8008F7D8093D8008091E0003D
:1046E00082608093E0008091E00081FDFCCF08951E
:1046F000AF92BF92CF92DF92FF920F931F93CF930F
:10470000DF936C01EB018A010E94D724F82E8111FE
:1047100023C00115110539F0F80180819181C81B72
:10472000D90BC80ED91EB12CA12C2097A9F08091CD
:10473000E80085FD22C08091E8008E778093E80034
:1047400001151105A1F0F80180819181A80EB91E13
:10475000B182A08285E0F82E8F2DDF91CF911F913D
:104760000F91FF90DF90CF90BF90AF9008950E947F
:10477000D7248823D1F2F82EEFCFF60181916F0173
:104780008093F1002197FFEFAF1ABF0ACECFFC0153
:104790008091EE029091EF0286179707A0F06115C5
:1047A000710529F49091E8009E779093E80090E0DD
:1047B0006115710551F4911108C08091E80082FFE4
:1047C00034C080E00895BC01F2CF8091E7028823D5
:1047D000C1F18530C1F18091E80083FD30C0809146
:1047E000E80082FDEACF8091E80080FFE1CF809170
:1047F000F3002091F200382F6115710519F028306F
:10480000310558F091E02830310509F090E0209111
:10481000E8002E772093E800CBCF81918093F100C0
:10482000615071092F5F3F4FE7CF8091E7028823E6
:1048300041F0853041F08091E80083FFBECF81E0F8
:10484000089582E0089583E00895FC018091EE02CE
:104850009091EF0286179707A0F06115710529F472
:104860008091E8008E778093E80090E061157105F3
:1048700051F4911108C08091E80082FF35C080E0BA
:104880000895BC01F2CF8091E7028823C9F18530F9
:10489000C9F18091E80083FD31C08091E80082FD7C
:1048A000EACF8091E80080FFE1CF8091F300209172
:1048B000F200382F6115710519F02830310558F0D4
:1048C00091E02830310509F090E08091E8008E7782
:1048D0008093E800CBCF84918093F10031966150B2
:1048E00071092F5F3F4FE6CF8091E702882341F0A7
:1048F000853041F08091E80083FFBDCF81E00895CD
:1049000082E0089583E00895982F973028F08F7003
:104910008093E90081E008959093E900242F762F99
:1049200050E0981731F07091EC002091ED0050911B
:10493000F00021FD02C09F5FE8CF3091EB003E7F89
:104940003093EB003091ED003D7F3093ED003091DE
:10495000EB0031603093EB007093EC002093ED009E
:104960005093F0002091EE0027FDE5CF80E0089500
:104970008091E80287FF13C08091E80082FF06C0A3
:104980008091E8008B778093E80004C08091E70273
:104990008111F2CF08958091E7028823D9F38091A5
:1049A000E80080FFF8CF8091E8008E77ECCF20916F
:1049B000E4003091E50095E6A9012091EC00822FFA
:1049C000817020FF06C08091E80080FF06C080E073
:1049D00008952091E80022FD1AC08091E702882303
:1049E00089F0853089F08091EB0085FD0FC0209122
:1049F000E4003091E50042175307F9F29150E1F6D7
:104A000084E0089582E0089583E0089581E00895A8
:104A10000E9477250E947F25E0EEF0E08081816092
:104A20008083E8EDF0E080818F77808319BCA7ED6B
:104A3000B0E08C918E7F8C9380818F7E80831092EA
:104A4000E60208950F931F93CF93DF930E9477257B
:104A50000E947F25C8EDD0E088818F778883888188
:104A60008068888388818F7D888319BC1092E702D3
:104A70001092E3021092E5021092E40200EE10E0C0
:104A8000F80180818B7F808388818160888342E008
:104A900060E080E00E948424E1EEF0E080818E7F7F
:104AA0008083E2EEF0E08081816080838081886095
:104AB0008083F80180818E7F8083888180618883F4
:104AC000DF91CF911F910F910895E8EDF0E0808183
:104AD0008F7E8083E7EDF0E080818160808384E0D9
:104AE00082BF81E08093E6020E9422250895E8EDCE
:104AF000F0E080818E7F80831092E2000895109212
:104B0000DA001092E10008951F920F920FB60F92F3
:104B100011242F933F934F935F936F937F938F93C2
:104B20009F93AF93BF93EF93FF938091E10082FF38
:104B30000BC08091E20082FF07C08091E1008B7F73
:104B40008093E1000E9446218091DA0080FF19C025
:104B50008091D80080FF15C08091DA008E7F80930D
:104B6000DA008091D90080FF96C080E189BD82E1A2
:104B700089BD09B400FEFDCF81E08093E7020E9469
:104B80000A218091E10080FF19C08091E20080FF3E
:104B900015C08091E2008E7F8093E2008091E20058
:104BA00080618093E2008091D80080628093D80079
:104BB00019BC85E08093E7020E942A218091E100E0
:104BC00084FF2BC08091E20084FF27C080E189BD73
:104BD00082E189BD89B5982F917080FFFBCF8091CC
:104BE000D8008F7D8093D8008091E1008F7E8093E4
:104BF000E1008091E2008F7E8093E2008091E200EC
:104C000081608093E2008091E302882309F449C027
:104C100084E08093E7020E9437218091E10083FFC6
:104C200029C08091E20083FF25C08091E100877F49
:104C30008093E10082E08093E7021092E30280918A
:104C4000E1008E7F8093E1008091E2008E7F80936F
:104C5000E2008091E20080618093E20042E060E047
:104C600080E00E9484248091F00088608093F000AE
:104C70000E942321FF91EF91BF91AF919F918F915E
:104C80007F916F915F914F913F912F910F900FBE48
:104C90000F901F90189519BC1092E7020E941C21DA
:104CA00070CF8091E30087FD93E09093E702B3CF4C
:104CB0001F920F920FB60F9211242F933F934F9391
:104CC0005F936F937F938F939F93AF93BF93CF9394
:104CD000DF93EF93FF93D091E900DF708091EC00B8
:104CE000C82FC17080FDC0E81092E9008091F000EB
:104CF000877F8093F00078940E949C261092E900B0
:104D00008091F00088608093F000CD2BCF70C0932D
:104D1000E900FF91EF91DF91CF91BF91AF919F910A
:104D20008F917F916F915F914F913F912F910F9054
:104D30000FBE0F901F901895AAE2B0E0E2EAF6E2EB
:104D40000C94332888EE92E02091F100FC0121932D
:104D5000CF01F2E0803F9F07B9F70E94A121809127
:104D6000E80083FF1EC18091E8029091E9029A3029
:104D700008F017C1E92FF0E0E453F74D0C941E281A
:104D8000803899F0823809F00CC18091EC028F7064
:104D9000873008F006C18093E9008091EB0085FB25
:104DA000882780F91092E90006C08091E402909172
:104DB000E502911182609091E800977F9093E8005E
:104DC0008093F1001092F1008091E8008E77E5C0A9
:104DD000882309F4D3C0823009F0E3C08091EA024D
:104DE0008111D6C08091EC028F702FEF280F2630F2
:104DF00008F0D7C08093E9002091EB0020FFC8C0E5
:104E0000933031F48091EB0080628093EB00C0C05E
:104E10009091EB0090619093EB0021E030E001C0B5
:104E2000220F8A95EAF72093EA001092EA00809117
:104E3000EB008860EACF8111B4C01091EA021F77BD
:104E40008091E3008078812B8093E3008091E800DB
:104E5000877F8093E8000E94B8248091E80080FF5B
:104E6000FCCF8091E30080688093E30082E0111121
:104E700083E08093E70295C08058823008F091C0AB
:104E80008091EA029091EB028C3D23E09207A1F51C
:104E900083E08A838AE289834FB7F894DE01139610
:104EA00020E03EE051E2E32FF0E050935700E49120
:104EB00020FF03C0E295EF703F5FEF708E2F90E010
:104EC000EA30C0F0C7968D939D932F5F243159F738
:104ED0004FBF8091E800877F8093E8006AE270E02E
:104EE000CE0101960E94C7238091E8008B778093C2
:104EF000E80057C0C096E7CF6091EC027091ED02D8
:104F0000AE014F5F5F4F0E940823BC01892B09F45B
:104F100048C09091E800977F9093E80089819A813A
:104F20000E942524E1CF8038E1F58091E800877F59
:104F30008093E8008091E3028093F10045CF8111D6
:104F400030C09091EA02923060F58091E800877F4E
:104F50008093E8009093E3020E94B8248091E302DA
:104F6000882311F084E005C08091E30087FDFACF2B
:104F700081E08093E7020E94872113C08091EA02BA
:104F8000813079F481E0933009F080E08093E5028C
:104F90001092E9008091E800877F8093E8000E94EA
:104FA000B8248091E80083FF0AC08091E800877FE1
:104FB0008093E8008091EB0080628093EB00AA96DA
:104FC000E3E00C944F28CF938091E7028823A1F06F
:104FD000C091E900CF709091EC00892F817090FD15
:104FE00080E8C82B1092E9008091E80083FD0E94C0
:104FF0009C26CF70C093E900CF910895991B79E06A
:1050000004C0991F961708F0961B881F7A95C9F758
:105010008095089597FB072E16F4009407D077FD2E
:1050200009D00E945B2807FC05D03EF4909581953D
:105030009F4F0895709561957F4F0895EE0FFF1F64
:105040000590F491E02D09942F923F924F925F9238
:105050006F927F928F929F92AF92BF92CF92DF9288
:10506000EF92FF920F931F93CF93DF93CDB7DEB7ED
:10507000CA1BDB0B0FB6F894DEBF0FBECDBF099481
:105080002A88398848885F846E847D848C849B84D8
:10509000AA84B984C884DF80EE80FD800C811B81E6
:1050A000AA81B981CE0FD11D0FB6F894DEBF0FBE15
:1050B000CDBFED010895AA1BBB1B51E107C0AA1F7C
:1050C000BB1FA617B70710F0A61BB70B881F991FA9
:1050D0005A95A9F780959095BC01CD010895FB01E3
:1050E000DC0104C08D910190801921F441505040A1
:1050F000C8F7881B990B0895F999FECF92BD81BD21
:10510000F89A992780B50895A8E1B0E042E050E010
:105110000C94B028262FF999FECF92BD81BDF89A44
:10512000019700B4021639F01FBA20BD0FB6F894EB
:10513000FA9AF99A0FBE08950396272F0E948B289A
:105140000E948A28252F0E948B28242F0C948B28BC
:105150000196272F0E948B280C948A28DC01CB0112
:10516000FC01F999FECF06C0F2BDE1BDF89A319677
:1051700000B40D9241505040B8F70895F894FFCF15
:105180000A090A093B093B09C809E4096A096A09CD
:10519000EF097B0A8A0A8A0AC026E826D127E82670
:0C51A000D1271B273C27D12793279F27EE
:1051AC007A02280850011E0A14018320A8208720A7
:1051BC0005210021862001E200E900EA00B500B6D5
:1051CC0000B700CD008301CC008A0192019401212B
:1051DC0002230224022502260227022A02B300B46B
:1051EC00006F007000818283E200E900EA00B500E4
:1051FC00B600B700CD008301CC008A019201940166
:10520C002102230224022502260227022A02B300CD
:10521C00B4006F0070008182836697C63435309578
:10522C0036323331F7F6F5F493929190943F3F3F39
:10523C00006D6B5F64656C6179006D6B5F696E749A
:10524C00657276616C006D6B5F6D61785F73706514
:10525C006564006D6B5F74696D655F746F5F6D6124
:10526C0078006D6B5F776865656C5F6D61785F73F7
:10527C0070656564006D6B5F776865656C5F7469FC
:10528C006D655F746F5F6D617800407B226C0AF115
:0A529C0009CF0974098D09A6090065
:00000001FF
